:100000000EC01DC06AC01BC01AC019C018C017C0DE
:1000100016C015C014C013C012C011C010C01124E6
:100020001FBECFE5D1E0DEBFCDBF10E0A0E6B0E05F
:1000300001C01D92A136B107E1F777D017C1E0CF1B
:10004000FC0188E88A95F1F78CEC90E00197F1F7D4
:100050002081262309F021E08CEC90E00197F1F754
:100060008081862309F022608CEC90E00197F1F703
:100070008081862309F024608CEC90E00197F1F7F1
:100080008081862309F028608CEC90E00197F1F7DD
:100090008081862309F020618CEC90E00197F1F7D4
:1000A0008081862309F020628CEC90E00197F1F7C3
:1000B0008081862309F020648CEC90E00197F1F7B1
:1000C0008081862309F020688CEC90E00197F1F79D
:1000D00088E88A95F1F7822F08951F920F920FB644
:1000E0000F9211242F933F934F935F936F937F93BE
:1000F0008F939F93AF93BF93EF93FF9386E390E02B
:1001000060E19EDF80936000FF91EF91BF91AF911E
:100110009F918F917F916F915F914F913F912F911F
:100120000F900FBE0F901F90189580E886BD16BCEB
:100130008BB780628BBFAC9A7894C19AB99AC09AF7
:10014000B89AC29ABA9A32E4809160008634A9F4CF
:1001500020E0C198822F932F9A95F1F78F5F8F3F00
:10016000D1F7C19A80E004C0932F9A95F1F78F5F81
:100170008217D0F32F5F2F3F61F7809160008634A4
:10018000B9F420E0C19AC098822F932F9A95F1F785
:100190008F5F8F3FD1F7C198C09A80E004C0932F42
:1001A0009A95F1F78F5F8217D0F32F5F2F3F51F7AA
:1001B000809160008634B9F420E0C09AC298822F02
:1001C000932F9A95F1F78F5F8F3FD1F7C098C29A1E
:1001D00080E004C0932F9A95F1F78F5F8217D0F3D8
:1001E0002F5F2F3F51F7809160008634C9F420E0E3
:1001F000C29AC098C198822F932F9A95F1F78F5F7A
:100200008F3FD1F7C29AC09AC19A80E004C0932F61
:100210009A95F1F78F5F8217D0F32F5F2F3F41F749
:10022000809160008634C9F420E0C29AC09AC19AD5
:10023000822F932F9A95F1F78F5F8F3FD1F7C29856
:10024000C098C19880E004C0932F9A95F1F78F5F12
:100250008217D0F32F5F2F3F41F7809160008634E3
:1002600009F472CFC29AC09AC19A6ECFF894FFCFA8
:00000001FF
